:100000000C9436000C944B000C944B000C944B0059
:100010000C944B000C944B000C944B000C944B0034
:100020000C944B000C944B000C944B000C944B0024
:100030000C944B000C944B000C944B000C944B0014
:100040000C944B000C944B000C944B000C944B0004
:100050000C944B004C696E6534004C696E6533003E
:100060004C696E6532004C696E65310011241FBE0B
:10007000CFE5D8E0DEBFCDBF10E0A0E6B0E0E4EB16
:10008000F2E002C005900D92A436B107D9F70E94A4
:100090004D000C9458010C9400000E942E0161E068
:1000A00081E00E94EF0086E690E00E94E00061E0BF
:1000B00082E00E94EF0080E690E00E94E00061E0B4
:1000C00083E00E94EF008AE590E00E94E00061E09A
:1000D00084E00E94EF0084E590E00E94E000FFCF02
:1000E000AD9A85E08A95F1F70000AD9885E08A9594
:1000F000F1F70000089580FF02C0AB9A01C0AB98F1
:1001000081FF02C0AA9A01C0AA9882FF02C0A99AE0
:1001100001C0A99883FF02C0A89A01C0A8980C94B6
:100120007000CF93C82F82958F700E947B008C2F18
:100130008F700E947B0087EC90E00197F1F700C080
:100140000000CF910895AF980E949100AF9A089552
:10015000863D59F168F4803B01F128F48A3009F1B9
:100160008D30F9F00895853BD1F0843CE1F008959D
:10017000843E59F028F48C3DD1F08F3D61F0089514
:10018000863F29F08C3F29F0089581EE08958FEE87
:10019000089585EF089582EE08958FED089584EE19
:1001A000089589E0089580E0089581E0089582E04F
:1001B00008950E94A800893011F00C9491000895D0
:1001C000CF93DF93FC018491EF012196882321F0E6
:1001D0000E94D900FE01F7CFDF91CF9108959FEFE4
:1001E000980F943080F46150643168F48250833009
:1001F00030F4E82FF0E0E05AFF4F808101C080E842
:10020000860F0C94A300089583E00E947B002FEFDB
:1002100080E792E0215080409040E1F700C000006C
:1002200083E00E947B0087E592E00197F1F700C030
:10023000000083E00E947B0087EC90E00197F1F7DB
:1002400000C0000082E00E947B0087EC90E00197F4
:10025000F1F700C0000088E20C949100A79AAF98D3
:10026000A59AAD98A69AAE98A39AA29AA19AA09A96
:100270002FEF84E39CE0215080409040E1F700C0E4
:1002800000000E94040188E00E94A30081E00E9417
:10029000A3008FE19EE40197F1F700C0000086E023
:1002A0000E94A3008CE00E94A30084E10C94A300B0
:0402B000F894FFCFF0
:0402B400C094D4001E
:00000001FF
